:400000000040002011000000C9030000C903000080B500AF00F0DCF980B584B000AF021CFB1D1A70204A3B1C0B3312781A701F4A3B1C0A3312781A700423013BFB6018E05C
:400040001B4B1868391C0B31FA68131C5B009B18C3185B780B70164B1868391C0A31FA68131C5B009B18C3189B780B70FB68013BFB60FB68002B0ADB0D4B1968FA68131CF1
:400080005B009B185B5CFA1D12789A42D8D9094B3A1C0B3212781A60074B3A1C0A3212781A60BD4604B080BDCCF1FF0FCDF1FF0FDC0000201CFF0B4020FF0B4080B500AF3F
:4000C000234B12221A603020FFF7A6FF214B224A1278D2B21A60052000F07CFC1F4B35221A6000F019FCFA235B00181C00F04EFC012000F021FC1A4B1A4A1A601A4B80226E
:40010000D2051A60194B1A4A1A601A4B194A126808218A431A60FA23DB00181C00F0B6FB154B181C00F056FC144B154A1A60154B154A1A60154B802212061A60144B8022D1
:40014000D2021A60134B40221A60BD4680BDC0463000104028FF0B40FDF1FF0F2CFF0B4004010B40060000800C020B407C002E406A2D00006CF02E40DC05000000030140AE
:40018000007FBB000000014040FF008008010B4000010B401C01014080B582B000AF72B6334B00221A60FB1D00221A7023E0FB1D1A78131C5B009B185B002E4A9B183B60E0
:4001C0003B681A78597809020A43997809040A43DB781B0613431A1C3B6819795B791B020B439BB2101C191C00F076F9FB1D1A78FB1D01321A70FB1D1B78012BD7D91E4A47
:400200001E4B101C191C00F077F91D4B1D4A1A601D4B03221A601D4B1D4A1A601D4B992212041A601C4B802292021A601B4B1B4A1278D2B202210A43D2B21A70184B184A15
:400240001278D2B23C218A43D2B214210A43D2B21A70124B114A1278D2B216210A43D2B21A70FFF72BFF00F087F9BD4602B080BD6CF02E40600A00006C0A0000840A000020
:4002800000000240300000EE00000440080004403200D80000500F4004500F4000700F4001700F4010B5064C2378002B07D1054B002B02D0044800E000BF0123237010BD12
:4002C000F000002000000000580A000008B5084B002B03D00748084900E000BF07480368002B03D0064B002B00D0984708BDC04600000000580A0000F4000020C800002033
:400300000000000080B500AF084B1B78012B07D1074B1B88181C00F0B7F9044B00221A70012000F0F7F9BD4680BDC046100100200E01002080B582B000AFFB1D00221A70AA
:4003400062B600F081F91C4B181C00F0EFF9FB1D1A781A4B5200D25A194B1A80194B00221A7000F01DF9031C002B24D1052000F00DFB00F015F9031C002B1CD1C04600F060
:400380000FF9031C002BFAD0FB1D1A78FB1D01321A70FB1D1B78062B02D9FB1D00221A70FB1D1A78054B5200D25A054B1A80054B01221A70D5E7D4E705030000CC0000205D
:4003C0000E0100201001002080B500AFFEE7C04680B586B000AF224B7B61224B3B61204B7B6135E03B691B68FB603B695B68BB603B699B683B6000237B600CE0FB681A68F1
:40040000BB681A60BB680433BB60FB680433FB607B6804337B607A683B689A42EED13B69DB683B6000237B6008E0BB6800221A60BB680433BB607B6804337B607A683B688A
:400440009A42F2D13B6910333B617B69013B7B617B69002BC6D100F0D1FAFFF76BFFFEE701000000BC0A000080B582B000AF154B144A126801218A431A6000237B600FE04D
:400480007B68032B04D8104B7A689200D35800E00E4B0F4A796889008B507B6801337B607B682F2BECD9FFF777FE0A4B00221A60044B044A126801210A431A60BD4602B079
:4004C00080BDC0460000104000000000C903000000000020C000002080B582B000AF786039607A683B68101C00211A1C00F0ACFABD4602B080BDC04680B586B000AF78608E
:40050000396000233B6100237B612EE07B699B007A68D3181B68BB603B1C0F33BA681A70BB68FF229343BB6017E03B695B003A68D3181B781A1CBB68D3183A695200396802
:400540008A1852781A703B6901333B613B1C0F331A783B1C0F33013A1A703B1C0F331B78002BE2D17B6901337B617B69052BCDD9BD4606B080BDC04680B500AF054B03227B
:400580001A60054B03221A60044B00221A60BD4680BDC0463000304030003140000E3F4080B500AF044B1B68DAB201231340DBB2181CBD4680BDC0460400044080B500AFE7
:4005C000104B8022D2041A600E4B0E4A12681A60002000F04BF80B4B0A4A12681A600A4B0C221A60012000F089F8084B31221A60FA235B00181C00F047F8642000F052F8D0
:40060000BD4680BD00012040240120402801204090B583B000AFFC1D00F0EFF8031C2370084B084A126801210A431A60FB1D1B78181C00F0E6F80120182100F041F8BD4607
:4006400003B090BD0000204080B500AF064B1B78002B04D1FFF7B2FF034B01221A70FFF7D7FFBD4680BDC0460C01002080B582B000AF7860034B7A681204120C1A60BD46A2
:4006800002B080BD0801204080B582B000AF7860034B7A681204120C1A60BD4602B080BD1401204080B582B000AF7860034B7A681204120C1A60BD4602B080BD0C01204084
:4006C00090B585B000AF786039603C1C0F3400F094F8031C2370084B3A687968081C9040021C1A603B1C0F331B78181C00F089F8BD4605B090BDC0460800204080B582B08A
:4007000000AF7860024B7A681A60BD4602B080BD3801204080B582B000AF7860024B7A681A60BD4602B080BD3001204080B582B000AF786000F04CF87B68181C00F008F8BB
:40074000032000F013F800F039F8BD4602B080BD80B582B000AF7860034A84237968D150BD4602B080BDC0460000002090B585B000AF021CFB1D1A700E23FB603C1C0B3440
:4007800000F03BF8031C23700A4B0A4A11680A4A1140FA1D1078FA68041C9440221C0A431A603B1C0B331B78181C00F02AF8BD4605B090BD10E400E0FF3FFFFF80B500AF3C
:4007C000024B802292021A60BD4680BD00E100E080B500AF024B802292021A60BD4680BD80E100E0000000000230800803D00138FDD1C046C046C0467047EFF3108072B6A2
:40080000704780F31088704780B500AF0B4B0B4A126801218A431A60094B094A126830218A4310210A431A60054B054A126807218A4301210A431A60BD4680BD00F02E4001
:4008400000FF2E4080B500AF0E4B0E4A126802218A431A600C4B0C4A126807218A4302210A431A60084B084A126830218A4320210A431A60034B034A126801210A431A6049
:40088000BD4680BD00F02E4000FF2E4080B584B000AF78600023FB60154B154A126801210A431A60134B144A1A60144B134A1268802109020A431A607B68002B13D010239A
:4008C000FB600DE0012000F085F800F019F8031C002B02D00023FB6005E07B68013B7B607B68002BEED1FB68181CBD4604B080BD60F02E4078002E400220000010002E400C
:4009000080B500AF034B1A6801231340181CBD4680BDC0460C002E4080B500AFFFF774FF044B044A1268802109060A431A60BD4680BDC04600F02E4080B584B000AF786029
:400940000C4B1A6801231340FB607B68002B02D0012B03D005E0FFF757FF06E0FFF772FF03E0002000F008F8C046FB68181CBD4604B080BD00F02E4080B582B000AF021C59
:40098000FB1D1A7001BEBD4602B080BD80B582B000AF786008E00C4B1B68181CFFF724FF7B680A4A9B187B607A6880231B029A42F1D8074B1B687A685343181CFFF714FF51
:4009C000BD4602B080BDC046EC0000200080FFFFE400002080B582B000AF021CBB1D1A80BB1D1B88044A12785343181CFFF7FCFEBD4602B080BDC046E800002070B50E4B40
:400A00000E4D0024ED1AAD101E1CAC4204D0A300F35898470134F8E700F03EF8084B094D0024ED1AAD101E1CAC4204D0A300F35898470134F8E770BDA40A0000A40A000079
:400A4000A40A0000AC0A0000031C8218934202D019700133FAE77047000000000400000000300F40000400400F40000401330F4002400F4002410F4002420F4001430F4077
:400A800002600F40EE085320D420AF20EE101280C408AE8002011101F8B5C046F8BC08BC9E467047CD02000069040000F8B5C046F8BC08BC9E467047A5020000D00A000071
:400AC000C800002028000000280000000000000000000000F401210258029A02EE025903E8030000C0F1FF0F006CDC0280BB0000300000000000C05D0000000000000000E8
:400B000000000000000000000000000000000000000000000000000000000000000000000000000000000000000000000000000000000000000000000000000000000000B5
:400B40000000000000000000000000000000000000000000000000000000000000000000000000000000000000000000000000000000000000000000000000000000000075
:400B80000000000000000000000000000000000000000000000000000000000000000000000000000000000000000000000000000000000000000000000000000000000035
:400BC00000000000000000000000000000000000000000000000000000000000000000000000000000000000000000000000000000000000000000000000000000000000F5
:020000040001F9
:0200000490303A
:020000009D441D
:0200000490402A
:4000000000000000000000000000000000000000000000000000000000000000000000000000000000000000000000000000000000000000000000000000000000000000C0
:400040000000000000000000000000000000000000000000000000000000000000000000000000000000000000000000000000000000000000000000000000000000000080
:0200000490501A
:0C00000000020E09119E00010E0CAEE281
:0200000490600A
:0100000001FE
:00000001FF
